:020000040000FA
:040000006FEF00F0AE
:0800080077D00D6E960E046E18
:10001000980E056E3DD8D8B4CA90D8A4CA80FC0FFB
:10002000D8A0CA92D8B0CA82800E046E960E056E11
:10003000980E086E096ACAB025D8CAB223D82AD841
:100040000404CB6E04C006F005C007F000500A6E31
:100050000B6E003C0B6A33D809500D2E0AD0BE6ED1
:100060000C0EBD6E08BEBD8A08BCBD889394CA84C0
:100070001200BB6E0C0EBA6E08BEBA8A08BCBA88F3
:100080009492F5D700D8D890083205320432120085
:10009000096A086A100EF36E0534083609360650F0
:1000A000085C0750095805E30650085E0750095AD6
:1000B000D88004360536F32EEFD7045012000650D0
:1000C0000A02F3CF08F0F4CF09F007500A02F35008
:1000D000092606500B02F350092608501200F86A50
:1000E0004F0EAF6E240EAC6E900EAB6E0001070E7D
:1000F000B46E0F0EC16E55D09EAA1BD0060EAB1467
:1001000012E1E1CF34F0E2CF35F0362A1EEE80F076
:100110003650E126000EE222AECFE7FF34C0E1FF09
:1001200035C0E2FF1100AE50AE50AB98AB88110065
:1001300006D0F2A404D0F294104A112A1100110042
:100140003650375C14E0372AE9CF04F0EACF05F0E7
:100150000EEE80F03750E926000EEA22EF50046ED2
:1001600004C0E9FF05C0EAFFD880120004D0E868A7
:10017000046ED8A012001200366A376A9D8AF28E89
:10018000F28C12009D9A0EEE80F0000EEE6AE82EC0
:10019000FDD7366A376A9D8A12009EA8FED7AD6EDB
:1001A0001200700E926EE00E936EC00E946E9396D7
:1001B0008A96929689969294899492928992929034
:1001C000899093988A9894948B9494928B92949615
:1001D0008B96336AD1DFD6DF170ED56ED76AD66A13
:1001E000F294F28AD58E06EC04F0AADF126EB20EFB
:1001F000125C07E3FE0E125C02E308D102D0146A1F
:1002000005D112AE21D0146A810E125C05E112C034
:1002100014F01568166817D0910E125C05E112C033
:1002200014F0176818680FD0A10E125C05E112C017
:1002300014F019681A6807D0B10E125C04E112C0FC
:1002400014F01B681C68E2D0145202E1DFD0DED04B
:10025000810E145CD8A442D0152803E112C015F019
:100260003BD012C016F03A0E155C08E1006A420E4F
:10027000066E0F0E076E010EC8DE2DD03B0E155C0C
:1002800003E194928B9227D06E0E155C05E13390BA
:100290002990929689961FD06F0E155C05E13392D6
:1002A00029929294899417D0700E155C05E13394CD
:1002B0002994929289920FD0710E155C05E13396C4
:1002C00029969290899007D0720E155C04E13398BC
:1002D000299893988A98156899D098D0910E145CB3
:1002E000D8A47BD0172803E112C017F074D012C035
:1002F00018F018523AE13A0E175C08E1006A420E13
:10030000066E0F0E076E010E80DE2DD03B0E175CC1
:1003100003E194928B9227D06E0E175C05E1339027
:100320002990929689961FD06F0E175C05E1339243
:1003300029929294899417D0700E175C05E133943A
:100340002994929289920FD0710E175C05E1339631
:1003500029969290899007D0720E175C04E1339829
:10036000299893988A98176851D03A0E175C0AE139
:1003700018501824006E420E066E0F0E076E010E06
:1003800044DE28D03B0E175C03E194928B8222D08E
:100390006E0E175C04E13380929689861BD06F0E37
:1003A000175C04E133829294898414D0700E175C38
:1003B00004E13384929289820DD0710E175C04E1BE
:1003C00033869290898006D0720E175C03E13388E1
:1003D00093988A8817681AD019D0A10E145C0AE184
:1003E000192803E112C019F003D012C01AF0B8D8CE
:1003F0000DD00CD0B10E145C09E11B2803E112C032
:100400001BF003D012C01CF0D4D900D02952D8B4AC
:10041000A1D029A01ED042C023F043C024F04CC07C
:1004200021F04DC022F010C031F011C032F0D6CF13
:100430002FF0D7CF30F021502F5C2250305823506E
:1004400031582450325832502418D8B0800AD8B8C5
:10045000F8D929A21ED044C023F045C024F04EC0D4
:1004600021F04FC022F010C031F011C032F0D6CFD1
:100470002FF0D7CF30F021502F5C2250305823502E
:1004800031582450325832502418D8B0800AD8B885
:10049000FAD929A41ED046C023F047C024F050C08A
:1004A00021F051C022F010C031F011C032F0D6CF8F
:1004B0002FF0D7CF30F021502F5C225030582350EE
:1004C00031582450325832502418D8B0800AD8B845
:1004D000FCD929A61ED048C023F049C024F052C040
:1004E00021F053C022F010C031F011C032F0D6CF4D
:1004F0002FF0D7CF30F021502F5C225030582350AE
:1005000031582450325832502418D8B0800AD8B804
:10051000FED929A81ED04AC023F04BC024F054C0F5
:1005200021F055C022F010C031F011C032F0D6CF0A
:100530002FF0D7CF30F021502F5C2250305823506D
:1005400031582450325832502418D8B0800AD8B8C4
:1005500000DA05D0010E115C02E3106A116A45D67B
:100560006E0E195C37E133A031D02980D6CF2FF041
:10057000D7CF30F010C031F011C032F01A1C036E2A
:100580007F0E03140E6E0F6A0EC002F0016AD8903F
:10059000023601C038F002C039F038C001F039C06D
:1005A00002F001502F24216E02503020226E000EE6
:1005B0003120236E000E3220246E23C042F024C06E
:1005C00043F021C04CF022C04DF003D02990929608
:1005D0008996E7D06F0E195C37E133A231D02982BA
:1005E000D6CF2FF0D7CF30F010C031F011C032F09D
:1005F0001A1C036E7F0E03140E6E0F6A0EC002F0FB
:10060000016AD890023601C03AF002C03BF03AC00D
:1006100001F03BC002F001502F24216E0250302027
:10062000226E000E3120236E000E3220246E23C075
:1006300044F024C045F021C04EF022C04FF003D05A
:10064000299292948994ADD0700E195C37E133A44D
:1006500031D02984D6CF2FF0D7CF30F010C031F071
:1006600011C032F01A1C036E7F0E03140E6E0F6A57
:100670000EC002F0016AD890023601C03CF002C000
:100680003DF03CC001F03DC002F001502F24216E2E
:1006900002503020226E000E3120236E000E3220D8
:1006A000246E23C046F024C047F021C050F022C081
:1006B00051F003D029949292899273D0710E195CF3
:1006C00037E133A631D02986D6CF2FF0D7CF30F0FF
:1006D00010C031F011C032F01A1C036E7F0E0314EB
:1006E0000E6E0F6A0EC002F0016AD890023601C089
:1006F0003EF002C03FF03EC001F03FC002F00150AA
:100700002F24216E02503020226E000E3120236EE5
:10071000000E3220246E23C048F024C049F021C0CE
:1007200052F022C053F003D029969290899039D08C
:10073000720E195C36E133A831D02988D6CF2FF05C
:10074000D7CF30F010C031F011C032F01A1C036E58
:100750007F0E03140E6E0F6A0EC002F0016AD8906D
:10076000023601C040F002C041F040C001F041C07B
:1007700002F001502F24216E02503020226E000E14
:100780003120236E000E3220246E23C04AF024C094
:100790004BF021C054F022C055F003D02998939813
:1007A0008A98196812001D6812001F6812001E68DE
:1007B0001200420E1B5C0BE11C5204E10ED8939612
:1007C0008A9602D093968A861CC02BF004D07B0EAA
:1007D0001B5CD8B402D81B681200296A92968996CD
:1007E00092948994929289929290899093988A98FF
:1007F00094928B9294968B96006A420E066E0F0E20
:10080000076E010E05EC00F0336A120093968A968B
:1008100092968996929489949292899292908990D4
:1008200093988A9894928B9294968B96006A420E33
:10083000066E0F0E076E010E05EC00F0296A336A92
:10084000120033B004D02990929689961BD029804B
:1008500038C001F039C002F001502F24216E02503F
:100860003020226E000E3120236E000E3220246EC6
:1008700023C042F024C043F021C04CF022C04DF010
:1008800080769296120033B204D029929294899481
:100890001BD029823AC001F03BC002F001502F2446
:1008A000216E02503020226E000E3120236E000E89
:1008B0003220246E23C044F024C045F021C04EF005
:1008C00022C04FF080749294120033B404D0299463
:1008D000929289921BD029843CC001F03DC002F065
:1008E00001502F24216E02503020226E000E312044
:1008F000236E000E3220246E23C046F024C047F041
:1009000021C050F022C051F080729292120033B692
:1009100004D02996929089901BD029863EC001F080
:100920003FC002F001502F24216E02503020226E71
:10093000000E3120236E000E3220246E23C048F0BA
:1009400024C049F021C052F022C053F08070929030
:10095000120033B804D0299893988A981BD029881C
:1009600040C001F041C002F001502F24216E02501E
:100970003020226E000E3120236E000E3220246EB5
:1009800023C04AF024C04BF021C054F022C055F0DF
:08099000817893981200FFD753
:020000040030CA
:0300010006170ED1
:020005008580F4
:060008000FC00FE00F40E5
:00000001FF
